:020000040000FA
:06000000AFEF26F0120034
:060008008DEF0BF0120069
:06002A000400AE4D0000D1
:100030004C01000046000000AA4D0000B402000080
:1000400004000000A64D0000B00200000400000003
:0C005000A44D0000FD00000002000000B4
:0800F8000001976B0101C369CF
:10010000C46B0101C16BC26BA10E0101BF6FC06B5B
:10011000E0EC17F00001806F12000401530EA86F8D
:100120004E0EA96F4D0EAA6F500EAB6F2E0EAC6F18
:10013000420EAD6F490EAE6F420EAF6FB06B80C016
:10014000C7F1D1EC18F0000901E1010C80C0D0F03A
:10015000ADEC07F000019F0EAD6F040EAE6F000115
:10016000970EAB6F040EAC6FF1D90401A46FE85089
:1001700038E00001A00EAF6F040EB06F23DA000963
:1001800030E0000197910201A80E896F040E8A6F7A
:10019000FDEC1CF0F3CFA5F4F4CFA6F40401F31C9E
:1001A00001E1A61D02E000019781A4C4B6F00001A0
:1001B000A00EB46F040EB56F9FC4B3F00001970E8C
:1001C000B16F040EB26F16DA0401A76F000197A198
:1001D00002D06BEC1DF00401A75103E072EC18F0A3
:1001E000010C02EC19F0010C9AC0E6FF9BC0E6FF7F
:1001F000810EE66E000EE66EA5EC24F0E552E552A7
:10020000E552E5529CC089F09DC08AF09EC08BF0FB
:100210009FC08DF0A0C08EF0A1C08FF0A2C090F062
:1002200098C06CF299C06DF25FEF25F00201000EEC
:10023000706F040E716FA3C06EF2A4C06FF275EC04
:1002400025F0000922E0A3C0E9FFA4C0EAFFEECF39
:1002500006F4EECF07F4EECF08F4EFCF09F4A20EC8
:100260000101C36FC46B0101000EC16F040EC26FA8
:100270000101FE0EBF6FC069E0EC17F000018C6F4A
:10028000FF0E8C5D01E1000C010C000C0401530E0B
:10029000346F4E0E356F4D0E366F500E376F2E0E7B
:1002A000386F420E396F490E3A6F420E3B6F3C6B0E
:1002B0000201340E896F040E8A6FFDEC1CF0F3CF3F
:1002C00032F4F4CF33F40401F31C03E1331D01E1F4
:1002D000E1D08CC0D0F0ADEC07F089C000F404018F
:1002E000810E306F000E316F0001300E2CEC0BF0E0
:1002F00091C026F492C027F475EC0BF00001D16B8D
:1003000079EC0AF000C4D1F0C0EC0AF00AE030C485
:10031000E9FF31C4EAFF302B000E3123EFCFD1F0DB
:10032000F3D70001A40E2CEC0BF091C028F492C07E
:1003300029F423EC0BF00001110ED76F040EA0EC92
:100340000AF08AC0D2F006EC08F0000901E1A0D062
:10035000040117AD9DD01CC48BF21DC48CF272EC4D
:100360001DF00001060E2CEC0BF083EC1DF00401D7
:10037000006F116FE8CFD1F0C0EC0AF005E083EC1C
:100380001DF00001D16FF8D793EC1DF00001400E75
:10039000D16F79EC0AF004C1D1F0BDEC07F005C1D2
:1003A000D1F0BDEC07F006C1D1F0BDEC07F007C1FC
:1003B000D1F034EC0AF00001060ED16F34EC0AF0F3
:1003C0008BC0D1F0BDEC07F00001430ED16F79EC8A
:1003D0000AF090C0D1F0BDEC07F08FC0D1F0BDECB9
:1003E00007F08EC0D1F0BDEC07F08DC0D1F0FAEC73
:1003F0000AF091C02AF492C02BF40001D16BFAEC00
:100400000AF091C02CF492C02DF423EC0BF0000103
:10041000100ED76F040EA0EC0AF0A5C0D2F006ECC7
:1004200008F0000935E00001060E2CEC0BF0040189
:100430001029F4EC0AF010C400F40401010E126F4C
:10044000040E136F04010051000700090AE012C4F2
:10045000E9FF13C4EAFF122B000E13234CEC0BF040
:10046000F1D7AAC0D1F0BDEC07F00001240EE46F73
:10047000040EE56F18C4E3F0CEEC08F0000908E0C4
:1004800024C4D1F0BDEC07F0FF0E0401255D07E1A7
:100490006BEC1DF08CC0C5F12EEC18F0000C25C4DF
:1004A00000F425C4D1F0C0EC0AF009E00051EA6A7A
:1004B000A60FE96E000EEA22EFCFD1F0F4D725297E
:1004C000010F1025020F010F006F91C02EF492C092
:1004D0002FF42CC491F02DC492F07EEC0AF0020EA1
:1004E000040100272AC491F02BC492F000C4D1F07B
:1004F000BDEC07F0020E04010025060F030F030FE9
:10050000060F1125020F006F28C491F029C492F044
:100510007EEC0AF0020E0401002500018925020F7D
:10052000030F0401006F26C491F027C492F07EEC03
:100530000AF02EC491F02FC492F06BEC1DF072EC17
:1005400018F08CC0C5F12EEC18F0010C0001080E5B
:10055000CE6F040ECF6F93EC07F0000901E1000CA1
:100560000001080EC46F040EC56FD7EC06F0000939
:1005700001E1000C0401085101E0000CADC0C2F023
:10058000AEC0C3F0ABC0C0F0ACC0C1F0E4DB00094A
:1005900001E1000C00010C0EC66F040EC76F16ECD3
:1005A00007F0000901E1000CABC02BF1ACC02CF14D
:1005B0000CC42AF19CEC0CF0000901E1000C0401D0
:1005C0000C51120090EC0AF0000911E0AFC0E9FFF5
:1005D000B0C0EAFF08C4EEFF09C4EEFF0AC4EEFF94
:1005E0000BC4EEFF90EC0AF0000902E1000C000CD5
:1005F00090EF0AF079EC0BF091C060F492C061F4D6
:1006000023EC0BF075EC0BF023EC0BF0B3C092F481
:100610000001040E2CEC0BF0B3C0D1F0BDEC07F0E0
:100620000001B351B30700090AE0B1C0E9FFB2C04D
:10063000EAFFB12B000EB223EFCFD1F0EFD70001CC
:10064000A20E6FEC0AF091C062F492C063F423EC46
:100650000BF023EC0BF00001020ED16F79EC0AF0E5
:10066000B4C0E9FFB5C0EAFF030E68EC0AF0020E61
:1006700068EC0AF0010E68EC0AF0EFCFD1F034EC30
:100680000AF091C064F492C065F475EC0BF091C06F
:1006900066F492C067F423EC0BF004015F6B5D6BB2
:1006A0005E6B0001590ECE6F040ECF6F93EC07F016
:1006B000000901E1000C79EC0BF091C068F492C0E4
:1006C00069F423EC0BF023EC0BF00401906B916BBD
:1006D00059515A1101E119D15F2B00015B0ECE6F08
:1006E000040ECF6F93EC07F00401586FE85001E15E
:1006F000000C5B51595F5C515A5B58510B6E0C6A90
:100700000B50595F0C505A5B79EC0BF091C06AF4B6
:1007100092C06BF423EC0BF023EC0BF000017B0E8A
:10072000CC6F040ECD6F00016C0ECA6F040ECB6F40
:10073000CDDB000901E1000CA30E0001B65D04E071
:10074000BCDB000901E1000C0001060E2CEC0BF0F3
:1007500091C093F492C094F47BC4D1F0BDEC07F047
:1007600004016C0E7C6F040E7D6F7BC458F4040191
:100770005851580700090AE07CC4E9FF7DC4EAFF2C
:100780007C2B000E7D234CEC0BF0F1D700017E0E8C
:10079000BC6F040EBD6F7BC4BBF000016C0EB96F63
:1007A000040EBA6FDFD9000929E1040153EC0BF004
:1007B000A30E0001B65D06E05EEC0AF0040E040133
:1007C0007B2587D0E9EC07F0F4EC0AF0E9EC07F0C0
:1007D0000401586F7EEC0AF0020E04017B25020F23
:1007E0008E6F8F6B040158515807000974E08E2BEF
:1007F000000E8F23EEDBF4EC0AF0F4D7A00E00011C
:10080000B65D25E1020E04017B258E6F8F6B14EC23
:100810000BF00001EC6B00017E0EEA6F040EEB6F33
:100820008BEC09F00401586FE85009E119EC0BF06A
:1008300053EC0BF05EEC0AF00401020E586F5851B5
:100840000B6E0C6A0B508E270C508F2344D0A10ED8
:10085000B65D22E114EC0BF093C491F094C492F0D5
:1008600000017E0EB76F040EB86F81D80401586F77
:10087000E85010E119EC0BF05FC4F2F00001020E39
:10088000F16F54EC0AF05EEC0AF0020E04017B25D5
:10089000020F1FD0020E1CD0A30EB65D1CE100019A
:1008A0005E0EE86F040EE96F00017E0EE66F040E27
:1008B000E76FEFEC08F00401586F5E5106E05FC48B
:1008C000F2F05EC4F1F054EC0AF0020E04017B2554
:1008D00058258E6F8F6B14EC0BF06AC491F06BC4CB
:1008E00092F08FC4D1F049DB8EC4D1F046DB040E08
:1008F00004010C6A8E250B6E8F510C220B50902731
:100900000C50912319EC0BF0E3D668C491F069C444
:1009100092F0C6EC0AF0040E04019025906F000ED0
:100920009121916F060E9027000E9123030E9027C0
:10093000000E9123030E9027000E912362C491F0C4
:1009400063C492F0C6EC0AF0050E04019225040F70
:100950009025906F000E9121916F60C491F061C459
:1009600092F07EEC0AF090C4D1F007DB010C040198
:10097000506B006B7DEC0BF0100B0FE17DEC0BF07E
:10098000040B040A01E0010E0B6E7DEC0BF0100B62
:10099000100A01E0010E0B140BE00401010E506F70
:1009A000B7C0BEF0B8C0BFF07BD9000901E1000CB0
:1009B0000001480EDD6F040EDE6F0001150EDB6FC7
:1009C000040EDC6FB7C0D9F0B8C0DAF055DB00090F
:1009D00001E1000C0401150E136F040E146F91C099
:1009E0004CF492C04DF448C400F4010E4C250001B3
:1009F000916F000E04014D210001926F040100511E
:100A0000000700090AE013C4E9FF14C4EAFF132B2E
:100A1000000E14234CEC0BF0F1D748C400F463EC47
:100A20000AF0040EEB50566F050EEB504B6F30EC96
:100A30000AF0040B1AE123EC0BF00401002BCDECBF
:100A40000AF0482BD6EC0AF0DEEC0AF00401026F43
:100A5000E85009E14EC491F04FC492F05EEC0AF008
:100A60000401020E026F02517AD0516B50050FE162
:100A70000101520E3D6F040E3E6F0101510E3B6F9E
:100A8000040E3C6F63EC0AF0ACEC0AF032E063EC6D
:100A90000AF0030E48EC0BF0EFCF4AF484C28BF25D
:100AA00085C28CF272EC1DF083EC1DF00401576BD3
:100AB00083EC1DF00401496F83EC1DF00401086F05
:100AC00083EC1DF00401076F63EC0AF00E0EEB508F
:100AD000116F93EC1DF00401505110E10101110E52
:100AE000376F040E386F08C436F139EC0DF0000989
:100AF00005E14CC491F04DC492F04FD70401069328
:100B0000069906850001010EEC6F0001030EEA6FE5
:100B1000040EEB6F8BEC09F00401572763EC0AF02D
:100B20000E0E11C4EBFF5751002757514827CDEC4B
:100B30000AF0D6EC0AF063EC0AF0030E48EC0BF076
:100B40004AC4EFFF63EC0AF0050E4BC4EBFF63EC05
:100B50000AF0040E56C4EBFFDEEC0AF00401002795
:100B600000511200000197A1000CEFEC0AF0F3CF46
:100B700003F4F4CF04F4BBC005F403C48BF204C443
:100B80008CF272EC1DF044EC0AF084C2EEFF85C2D8
:100B9000EDFF83EC1DF00401026F80EC0BF0030EFF
:100BA0003CEC0AF050EC0BF0800B05E080EC0BF015
:100BB000050E3CEC0AF050EC0BF0080B02E032ECB6
:100BC0000BF01EEC0BF0EF500401025D16E000018B
:100BD000BB510401055D3AE050EC0BF0080B5DE001
:100BE00093EC1DF000C490F201C491F2DAEC1DF018
:100BF000F3CF03F4F4CF04F4C0D705070001B92BF9
:100C0000000EBA2350EC0BF0100B10E150EC0BF07F
:100C1000010B02E032EC0BF080EC0BF0040E3CEC2C
:100C20000AF044EC0AF006EC0BF010D004010505C4
:100C300004E11EEC0BF0EF5009E0055107E084C21F
:100C400003F485C204F493EC1DF097D793EC1DF0E8
:100C50001EEC0BF0EFCF02F444EC0AF00E0E02C4CF
:100C6000EBFF040105510AE144EC0AF00E0E48ECDA
:100C70000BF0EF6883EC0BF0EF6A010C05510108F3
:100C800003E3800E021504E083EC0BF0EF68000C28
:100C900083EC0BF0010EEF6E010C93EC1DF0000CD9
:100CA0002FEC0BF0100B0DE12FEC0BF0080B04E117
:100CB0002FEC0BF0010B04E0E2DBB8EC0AF001D002
:100CC000000CDDDB84C2EEFF85C2EDFFD8DB68ECF3
:100CD0000BF05BEC0BF0020ECFDB5BEC0BF0030ECA
:100CE000CBDB2FEC0BF0800B04E05BEC0BF0050E84
:100CF000C3DB2FEC0BF0080B04E12FEC0BF0010B26
:100D00000FE083EC1DF00401B16F83EC1DF00401D2
:100D1000B26FB5DB0A0EB1C4EBFF0B0EB2C4EBFF32
:100D20002FEC0BF0100B03E093EC1DF0CAD75BEC3B
:100D30000BF0040EA1DBA3DB06EC0BF0A0DBF7EC61
:100D40000AF0010EEF6E9BDB0E0E48EC0BF0EF6A23
:100D500093EC1DF0010C3DD90401006F040E005D01
:100D600001E0000C36D90401016FC2C0E9FFC3C025
:100D7000EAFFEF6E0151080801E2000C0401015185
:100D8000010700090EE025D90401006F0001C0C071
:100D9000E9FFC1C0EAFFC02B000EC12300C4EFFF72
:100DA000EDD7C0C0E9FFC1C0EAFFEF6A010C040142
:100DB000046B056B066B076B0CD9020801E0000C95
:100DC0000001040EC86F040EC96F4AD8000901E182
:100DD000000C040ED88004010455000E0555000EC9
:100DE0000655000E075501E2000C006B016B026B0B
:100DF000036B0451040700090CE0EBD8E66E040114
:100E00000451EA6A000FE96E040EEA2264EC0BF06A
:100E1000F0D7C4C0E9FFC5C0EAFF00C4EEFF01C4BB
:100E2000EEFF02C4EEFF03C4EEFF010CD2D80401B2
:100E3000006FA00E005D07E0A10E005D04E0A30EB0
:100E4000005D01E0000CC6C0E9FFC7C0EAFF00C4B6
:100E5000EFFF0001010EC86F040EC96F30EF07F0FD
:100E600004010E6B0F6B106BB4D804010D6F0E6F85
:100E70000DAF17D00D9F0D51020801E2000C0D2996
:100E8000106F0D510D0700090EE0A3D8E66E0401A6
:100E90000D51EA6A0E0FE96E040EEA2264EC0BF0C3
:100EA000F0D7010E106FC8C0E9FFC9C0EAFF0EC439
:100EB000EEFF0FC4EDFF105112008BD8050801E0C2
:100EC000000C87D8000901E0000C010C82D806084C
:100ED00001E0000C0001000EC86F040EC96FC0DFF6
:100EE000000901E1000C04010F0ED8800055000E2E
:100EF000015501E2000CCCC0E9FFCDC0EAFF00C4FF
:100F0000EFFF04010051000700090CE062D8E66E13
:100F10000001CAC0E9FFCBC0EAFFCA2B000ECB23F9
:100F2000D3DBEFD7010C55D8300801E0000C0001ED
:100F3000000EC86F040EC96F93DF0401046FE85000
:100F400001E1000C042BCEC0E9FFCFC0EAFF00C4D2
:100F5000EEFF01C4EDFF04511200D0C0BEF140EC21
:100F600012F00009FAE0D5C195F0D6C196F0000163
:100F7000936B946B916B926B12000101BE51160D35
:100F8000F3CFE9FFF4CFEAFF920EE926010EEA2241
:100F9000130E7EDB91C0EEFF92C0EDFF080E000144
:100FA00091250101F46F000E000192210101F56FFE
:100FB000140EF427000EF52396C0F3F172EC14F032
:100FC000D1C0C6F132EC18F00001912B000E922333
:100FD0001200000193C0F1F194C0F2F1932B000EC6
:100FE0009423080E0101F127000EF223140EF127BD
:100FF000000EF2235FEC14F00101110EC86F040E15
:10100000C96FDBEC18F0040111511200E8DAF3CFDC
:101010003DF4F4CF3EF4D3C0E1F0D4C0E2F03DC4DF
:10102000DFF03EC4E0F086D849DB100B1FE146DB61
:10103000800B14E07CDA050EEB500001D25D0EE16E
:10104000D7C0DDF0D8C0DEF0D5C0DBF0D6C0DCF014
:10105000D3C0D9F0D4C0DAF03CEF08F02FDB080B96
:1010600003E12CDB010B07E062DA82DA84C23DF493
:1010700085C23EF4D0D7000CB2DAF3CFB3F4F4CF8C
:10108000B4F4D9C0E9FFDAC0EAFFEECFB1F4EDCF96
:10109000B2F40401C86BC76B0001B70EE16F040E18
:1010A000E26FB3C4DFF0B4C4E0F044D80401C75128
:1010B0000001EA6ADB25E96EDC51EA22B9C4EFFFE0
:1010C0000401B351B1190BE1B451B21908E1C72BB6
:1010D000DDC0E9FFDEC0EAFFC7C4EFFF010CC85165
:1010E000010A1FE0010AD8E1BAA719D0C1C4B5F4BA
:1010F000C2C4B6F4C1C490F2C2C491F2DAEC1DF0DD
:1011000084C2B5F485C2B6F40401B551B15DB651DF
:10111000B25905E3B5C4B3F4B6C4B4F4BDD7010EF7
:10112000C86FBAA9000CC72BC3C4B3F4C4C4B4F4C9
:10113000C86BB2D7DFC08BF2E0C08CF272EC1DF04E
:10114000D3D9DFC0EEFFE0C0EDFFBBDA020E94D9C9
:10115000B8DA030E91D9C8D9030EEB500401C96F58
:10116000C9AF03D0AEDA050E87D90401C9B785DA55
:10117000C9A906D0B9D90C0E84C2EBFF0D0E0AD056
:10118000C9B17BDA9EDA040E77D9AED9080E84C2D3
:10119000EBFF090E85C2EBFF93EF1DF00A0E000175
:1011A000E76EE319E8AE02D0E73402D0E750E35D22
:1011B00001E3000CE3C0F6FFF76AF6BEF7688EDACB
:1011C00005DA82DAE3C0F6FFF76AF6BEF76886DA78
:1011D000F722F62A000EFAD9EE5276DA010C040153
:1011E000006B0B6B34DA3CD9100B08E130DA38D9DC
:1011F000020B04E12CDA34D9200B02E1020E006F5D
:10120000E8DE0401036F82DA0001010EE46F040ED0
:10121000E56F1DDA040EEB500001E36FBFDF00093C
:1012200003E10401030E006F04010151035D02E0BC
:10123000030E006FCEDE0401046F68DA04517F08EC
:1012400002E2030E006F03DA0BD9040B07E1FFD9AA
:101250000E0EEB50000902E0020E006F056B066BEC
:10126000076B086B096BFF0E025D24E00451040854
:101270001EE304510407000911E0ABDE04010A6F0C
:101280000451EA6A050FE96E040EEA220AC4EFFF70
:101290000AC4D1F072DE04010B2BEBD7005132E10E
:1012A00031D909C431F1F5D800092CE10401030E4C
:1012B000006F28D004C42EF1CAD9050EEB500101ED
:1012C0002D6F9DEC0CF0000903E10401030E006F8B
:1012D00004010451040700090FE07BDE0401056FDF
:1012E00015DA0051F5E10ED90951092B0101316FD1
:1012F000D0D80009EDE1E9D7005104E103D901019B
:101300003169C7D8E8C0E9FFE9C0EAFF00C4EFFFD0
:1013100004010B5112000401C76BC86BC96BCA6B87
:10132000F9D9100B01E0000CF5D9040B06E1F3D854
:101330000E0EEB50000801E2000CEDD8040EEB504D
:10134000CC6F0001CD0EE46F040EE56FCCC4E3F06A
:1013500025DF000901E1000C0001EC510AE1CDC4D8
:10136000D1F00BDE91C0CFF492C0D0F4CEC4D1F056
:1013700004DED0D9020B15E0CED8080E89D9A8D941
:1013800083EC1DF00401CB6FC66F0401C651C60784
:10139000000904E083EC1DF027D9F7D793EC1DF08A
:1013A00030D00401C56BC76BC86BC96BCA6BCB6B04
:1013B0000101C70E3D6F040E3E6F0101C50E3B6F6C
:1013C000040E3C6FA8D8C8D81BE0FF0E0401CE5D08
:1013D0000EE0CEC4CBF40401CE5113E0CE07CE51C3
:1013E000EA6AC70FE96E040EEA2256D9F4D7CB2B6E
:1013F000C7C4D1F0C2DDFF0E0401C55DD9E101D043
:10140000000C0001EC5112E191C0D1F492C0D2F471
:10141000CFC491F0D0C492F0CBC4D1F0AEDDD1C432
:1014200091F0D2C492F00401CB2BCB2B0401CB5111
:10143000120091C000F492C001F4EDC091F0EEC032
:1014400092F0F1C0D1F099DDEFC091F0F0C092F0D0
:10145000F2C0D1F092DD00C491F001C492F012000C
:10146000030E16D9EF50120088DD0001020EF4D8E9
:101470000001010E2CEF0BF00BD964EF0BF0BEC096
:10148000E9FFBFC0EAFF1200BCC0E9FFBDC0EAFF30
:101490001200DDD80E0EEB500101306F050EEB503F
:1014A00001012F6FACEF0CF066C4EFF067C4F0F0F1
:1014B00064C4EDF065C4EEF019EF0AF00001050E0A
:1014C000CBD823EF0BF0B7C0E9FFB8C0EAFF12009A
:1014D000DFD8E2D8B4C0E9FFB5C0EAFF1200BCD83B
:1014E0000001820E2CEF0BF0E1C0E9FFE2C0EAFF41
:1014F000120043DD0001040E2CEF0BF0E8CFD1F019
:10150000BDEF07F005C432F106C433F107C434F16E
:1015100008C435F11200EAC0E9FFEBC0EAFF12008F
:101520000001080EC46F040EC56FD7EF06F0D3C0DC
:10153000E9FFD4C0EAFF120083EC1DF0E66E120052
:10154000D86F0001010ED56F040ED66F0001140E86
:10155000D36F040ED46F12000E0EEB5001013A6FE0
:10156000050EEB500101396F58EC0DF00009120027
:101570000A0E8ED8EECF90F2EDCF91F2DAEF1DF099
:10158000FCDC0401005100070009120091C4D1F0F5
:10159000F4DC90C4D1F0BDEF07F091C04EF492C0DE
:1015A0004FF44CC491F04DC492F0120048C4D1F0F5
:1015B000E4DC4EC491F04FC492F012000001EC6BD9
:1015C000B7C0EAF0B8C0EBF08BEF09F0F7220800E3
:1015D000F550E66EE4C0E9FFE5C0EAFF1200020143
:1015E000906B916BDAEF1DF000012CEF0BF00F0EFA
:1015F00048EF0BF0C2DC0001300E2CEF0BF00A0EAE
:1016000000C4EBFF0B0E01C4EBFF1200080E84C2F6
:10161000EBFF090E85C2EBFF12000A0ECAC4EBFFF6
:101620000B0ECBC4EBFF120091C095F492C096F460
:10163000120095C491F096C492F01200B9C0E9FF6F
:10164000BAC0EAFF12000001D16BBDEF07F0E6C09F
:10165000E9FFE7C0EAFF1200D16FBDEF07F00FDF2F
:1016600030EF0AF083EC1DF00401006F83EC1DF0F5
:101670000401016F09DFFFEF0AF083EC1DF00401A4
:10168000CA6F83EC1DF00401CB6F2EDF0DEF0BF062
:10169000E926000EEA221200EFCFD1F0BDEF07F0ED
:1016A000F3DE30EF0AF0020E5E6F5FC4F2F000016D
:1016B000F16F54EF0AF040DF3FEF0AF038DF30EF10
:1016C0000AF03ADF74EF0AF0E552E750EF6E1200CD
:1016D000EECF8BF2EDCF8CF272EF1DF0D890F63694
:1016E000F736900EF6264D0E12000001D16B34EF46
:1016F0000AF00001300E6FEF0AF0E5DE30EF0AF07D
:101700001BDF44EF0AF0C0DEF7EF0AF0F7DE04015A
:0A1710000B2B120000DF30EF0AF08F
:06171A00DACFE4FFE2CF8C
:10172000DAFFE9CFE4FFEACFE4FF00EE0BF0080EAA
:10173000E80403E3EECFE4FFFBD7E65292EC26F099
:10174000E55200EE12F0080EE80403E3E5CFEDFFEA
:10175000FBD7E5CFEAFFE5CFE9FFE5CFDAFF1100E0
:10176000ACA2FED721C1ADFF1200010122C1E9FFE9
:1017700023C1EAFF222B000E2323EFCF08F4EF5002
:1017800004E008C421F1ECDFF0D71200A1DA7BEC11
:1017900026F0F4EC1CF0B8DA81BA0BD026EC11F08C
:1017A0000201760EAD6F420EAE6F3BEC24F002EC00
:1017B00010F028EC22F07CEC00F001011CA10AD012
:1017C00026EC11F00201650EAD6F420EAE6F3BECE0
:1017D00024F006D00101010E7A6F0201070EB06FEE
:1017E00084EC26F001017B51045C0B6E7C510558A2
:1017F0000C6E7D5106580D6E7E512BEC11F00BE3F3
:1018000084EC26F004C07BF105C07CF106C07DF1BC
:1018100007C07EF1897831EC22F08DEC00F008DA17
:1018200001017A510201B35DDBE00101010E416F5C
:101830000101040E3F6F010E406FD8D9B3C27AF197
:1018400001011CA1CDD70201CE0EAA6F02EC24F03B
:101850000A0E01017A5D02E2300E01D0410E7A25B6
:101860000201AF6F4DEC24F0BBD70101245188EC8D
:1018700011F0030E0BEC11F0EFCF4FF4245188EC74
:1018800011F0020E0BEC11F0EFCF50F4245188EC64
:1018900011F0010E0BEC11F0EFCF51F4245188EC54
:1018A00011F0EFCF52F401017F51010A2AE0010A41
:1018B00042E184EC26F004C09FF005C0A0F006C011
:1018C000A1F007C0A2F00001060E9E6F00019D6905
:1018D00001012451D3EC10F0EFCF9CF02451D3EC54
:1018E00010F0EE52E9CF9AF0EACF9BF000014F0ED4
:1018F000986F040E996FF4EC00F00101010E7F6FF8
:10190000000C00014F0EA36F040EA46F16EC01F043
:10191000000911E001017F6B0001AA6B26C1A6F04E
:1019200027C1A7F028C1A8F029C1A9F025C1A5F0B9
:1019300046EC01F0010C000C010C01012D510A0ACA
:1019400006E00E0A08E1090E2E5D05E2010C110EFB
:101950002E5D01E2010C000C01012F510A0A6CE01E
:101960000E0A4EE0060A31E0010A17E0050A0AE015
:10197000030A01E07DD03251010BF36EF346F346CA
:10198000FB0E07D03251010BF36EF346F346F346DC
:10199000F70E8914F310896E010C59EC11F006E270
:1019A000305188EC11F04BEC11F0010C020E305D5F
:1019B0005FE2305188EC11F04BEC11F03051D3EC78
:1019C00010F0EF6A01015D2B010C59EC11F00FE2F0
:1019D000320505E130518CEC11F0EF80010C3251F1
:1019E00005E130518CEC11F0EF90010C000C020E6F
:1019F000305D3EE201015D2BADEC11F0EF6A000CB1
:101A0000FF0E315D09E159EC11F002E101015D2B9E
:101A1000ADEC11F0EF2A010C59EC11F029E2305134
:101A2000C2DBEE5231516AEC11F032C1EFFFADEC86
:101A300011F031C1EFFF010CFF0E315D0BE03151B0
:101A4000EA6A4C0FE96E010EEA2232C1EFFF010192
:101A50005C2B010C54EC11F063EC11F054EC11F020
:101A600002014C0EAB6F010EAC6F2AEC24F0010C9E
:101A7000000C7EEC11F0EFCFB1F401013651010AF8
:101A800016E101015D5101E1000CFF0E0401B15DA1
:101A900004E17EEC11F0EF6A010C01015D05040127
:101AA000B15D05E2B1297EEC11F0EF6E010C000C86
:101AB00083EC11F0EFCFB1F4010139510A0A01E1D1
:101AC0007AD00E0A5EE0070A46E0010A3CE0030A0B
:101AD00033E0080A2AE0010A21E00F0A1AE0010AAD
:101AE00014E0030A0EE0FF0A01E07FD084EC26F048
:101AF00004C00BF005C00CF006C00DF007C00EF0DE
:101B000036D08950040B25E007D08950080B21E01E
:101B100003D08150200B1DE0010E1BD090EC11F082
:101B200000C1EEFF01C1EDFF010C90EC11F002C10C
:101B3000EEFF03C1EDFF010CC1DB57E290EC11F0A9
:101B40003AC1EFFF010CBADB50E23A51E5DBEF504E
:101B5000010B76DB010CB2DB48E23A51D9DBEECF68
:101B60000BF0EECF0CF0EECF0DF0EFCF0EF0D8DB98
:101B70000BC0EEFF0CC0EEFF0DC0EEFF0EC0EEFF7F
:101B8000010C9CDB32E23A510EDBEF5011E03A518E
:101B90000ADBEE520401B1519DDBEF5051DB040131
:101BA000B12B01013A51FFDAEF500401B15D19E1A7
:101BB000AADBEF68010C01015C5103E10401B1698A
:101BC00010D00401B151B12BEA6A4C0FE96E010E3D
:101BD000EA22EF5035DB01015C510401B15D01E106
:101BE000B16991DBB1C4EFFF010C000C010141515F
:101BF00002E02CDB68DB2ADB05DBDFDA02E0F7DA68
:101C000001D0FBDAFFDA010EACDB02E0F0DA01D042
:101C1000F4DAF8DA020EA5DB02E0E9DA01D0EDDA57
:101C2000F1DA030E9EDB02E098EF11F09FEF11F066
:101C30008150200B05E10101805102E1010E806F0E
:101C400001015D51815D02E1816B806B80511BE080
:101C5000815162DBEF50010B15E00401536B53C45B
:101C600026F154C427F155C428F156C429F10101C5
:101C7000070E256F81C124F1F8DD000904E00101A0
:101C8000812B01D0812B810EC26E0101640E006F89
:101C9000005100070009FCE1C284C2B4FED7C3CFE3
:101CA00000F1C4CF01F1840EC16E890EC26E010134
:101CB000640E026F025102070009FCE1C284C2B443
:101CC000FED7C3CF02F1C4CF03F18E0EC16E120056
:101CD0008E0EC16E030E926E809A89848986F19E63
:101CE000D8EC23F0E1DA0201580EAD6F420EAE6F70
:101CF0003BEC24F0200EAC6E900EAB6E0F0EAF6E70
:101D0000D56AF28EF28C120001010A0E046F056F83
:101D1000050E066F0F0E076F0E690F691069116BC4
:101D20000A0E126F136F050E146F0F0E156F086BEE
:101D3000040E096FA30E0A6F0B6B0C6B0D6B1C81ED
:101D40000401040E046F010E056F0201776BC9DAFE
:101D5000A3EC1FF00401036FACEC1FF0550E04015F
:101D6000035D1BE1010E0201776FBBDA0401036B17
:101D70000351BDDA10E2A3EC1FF0E66E040104C4C7
:101D8000E9FF05C4EAFF042B000E0523E552E750E6
:101D9000EF6E032BEDD7ACEF1FF0CFEF0EF0040189
:101DA000040E016F010E026F0201746B756B02016C
:101DB000A00E736F22EC1FF00201550E796F85ECB7
:101DC0001FF00401006B005192DA0EE201C4E9FF3A
:101DD00002C4EAFF012B000E0223EFCF79F285EC5B
:101DE0001FF00401002BEFD799EF1FF0010142C152
:101DF000F6FF43C1F7FF422B000E43230800F5CF47
:101E000000F4F55004E000C421F1AADCEFD7120081
:101E10000401016B9EAAFED7AECF00F40D0E0401A3
:101E2000005D17E00A0E005D14E0012B010144C1C2
:101E3000E9FF45C1EAFF442B000E452300C4EFFF34
:101E400044C1E9FF45C1EAFFEF6A46514607000970
:101E5000E1E104010151120047C101F448C102F45B
:101E60000401036B47C1E9FF48C1EAFFEFCF00F46B
:101E7000EF5021E02E0E0401005D11E1010147C188
:101E8000E9FF48C1EAFF472B000E4823EF6AC7D994
:101E9000032BF7D947C101F448C102F407D0300E33
:101EA000005D03E30051390801E2000C0101472BFA
:101EB000000E4823D7D7B3D9E4D9030E0401035D3C
:101EC00001E0000C010C9EAAFED7AECF00F4310E4B
:101ED0000401005D05E3390E005D02E200511200CD
:101EE000390C01010D0E21DA01010A0E1EDA300E45
:101EF00001014B5DFF0FE96EEA6AD890E936EA36D8
:101F0000820EE926010EEA22EECF42F1EDCF43F137
:101F10006DDF01014B51380A73E00F0A6FE0010ACF
:101F20006BE0030A67E0010A35E0070A2EE0010AC8
:101F300027E0030A01E012008F0EE66E040EE66E43
:101F400016C1E6FF17C1E6FF01DA01018F0E226F0D
:101F5000040E236FB5EC0BF037D9000935E08F0E76
:101F6000E66E040EE66E08EC1EF0E552E552F3CF85
:101F700016F1F4CF17F1F4CF0CF1F3CF0DF11200FD
:101F80000401040EA76F010E09D00401120EA76F01
:101F9000010E04D004010E0EA76F010EA86F0101FF
:101FA000416BA7C43FF1E8CF40F120DE0DD901011C
:101FB000A30E496F040E4A6F01018F0E476F040E86
:101FC000486F4ADF000909E10101050E426F440E26
:101FD000436F0CDF9EBA0DD0FDD7A7C4E9FFA8C49C
:101FE000EAFFA3C4EEFFA4C4EEFFA5C4EEFFA6C49F
:101FF000EEFF12001C8112001C91120016EF10F06F
:10200000CFEF0EF00101960E426F420E436FEEDEEF
:102010005ADF0401AA6F390EAA5D03E0AAC44BF18E
:1020200060DF380E0401AA5DEDE112000401006BCF
:10203000046B96EC1DF0F3CF02F4F4CF03F416D941
:1020400092EC26F084EC26F004C08BF405C08CF4EE
:1020500006C08DF407C08EF4870EE96E040EEA6E9A
:10206000EE500401045C0B6EEE5005580C6EEE5001
:1020700006580D6EEE50EFD805E3F8D80101150EA5
:1020800054D989749EAADCD70401045101E076D0AA
:1020900092EC26F09EAAF8D78974AECF01F4040121
:1020A0000051030A21E0010A1CE0030A15E00105C2
:1020B00002E1010E17D0040E015D0AE189846BEC88
:1020C0001DF00101060E31D90401010E046FDCD7A9
:1020D0000101150E2AD9D8D7060E066F056B020E20
:1020E00001D0030E006FD0D70551052BEA6A070F08
:1020F000E96E040EEA2201C4EFFF05510B6E0C6A73
:102100000C50000AE8AE02D00C3405D0800ED88006
:102110000B54000E0C54B8E202C48DF203C48EF2CC
:102120009EEC1DF00401060E066F016B01510B6E53
:102130000C6A0C50000AE8AE02D0D89004D0800E91
:102140000B5C000E0C580DE20151EA6A070FE96EB4
:10215000040EEA22EFCF8FF2B4EC1DF00401012B44
:10216000E5D7CEEC1DF0F3CF02F4F4CF03F406C4B0
:1021700021F1B0EC0BF00401006B86D7010C4B0E83
:10218000E66E9FEC26F0E5521200140EE66E9FEC10
:1021900026F0E5521200F29E050EE66EBDEC26F02A
:1021A000E552F28E12000E0DF3CFE9FFF4CFEAFFF5
:1021B0005E0EE926010EEA221200EF50E66EE66A94
:1021C000C5D80101415112000101290EAED801010B
:1021D0003A0EABD80101200EA8D80101140E466FAB
:1021E00001018F0E446F040E456F08EF0FF0A0D869
:1021F00002012E0EAF6F4DEF24F0A1D801012E0E7B
:1022000095EF11F0000EE66E040EE66E3FC1E9FF99
:1022100040C1EAFF1200E926000EEA22120001C4C2
:10222000E6FF02C4E6FF08EC1EF0E552E552F3506B
:10223000E66E49C10BF04AC10CF0040103511200D3
:10224000E66E6ED8E552E750EF6E12000201C00E46
:10225000AA6F02EF24F007580E6E320E0B5C000ED0
:102260000C58000E0D58000E0E58120084EC26F08B
:1022700004C087F405C088F406C089F407C08AF456
:1022800012000F010B24E96F000E0C20EA6FE552DB
:10229000E750EF6E120032C1EEFF33C1EEFF34C1E2
:1022A000EEFF35C1EEFF12000201800EAA6F02EFB1
:1022B00024F001015D510101305D120001015D5109
:1022C00001013A5D12000201850EAD6F420EAE6F44
:1022D0003BEF24F00F01E924E96F000EEA20EA6FDA
:1022E0001200786B0201A00E766F58EF1FF00B6E94
:1022F0000C6A1D0E0B5C000E0C58120037C1E9FF72
:1023000038C1EAFF12003BC1E9FF3CC1EAFF1200FD
:102310004ADF090E0BEF11F046DF0D0E0BEF11F047
:102320003DC1E9FF3EC1EAFF1200216FB0EF0BF0A3
:102330000201000EAB6F040EAC6F2AEF24F0010116
:10234000000E226F040E236FB5EF0BF07DEC1EF034
:10235000E552E552E552E552120001013051D3EF4A
:0823600010F059DFDDEF10F071
:082368000401006B0051FEDAD4
:1023700015E20051040DF3CF0BF0F4CF0CF0400E3A
:102380000B26000E0C220051D1DA0BC0EFFF0051DA
:10239000CDDAEE52010EEF6E002BE8D70101D66BBD
:1023A00047DADEDA01011F0E0EDB0101EC6F0101DD
:1023B0001F0ECBDAD5DACCDA800B61E00101210EF9
:1023C000BFDACEDA0101480EEC6F01010E0EBDDA64
:1023D000C3DAD8DA040EEC6F01010C0EB6DA010193
:1023E000F5DADCDA440EEC6F0101010EAEDA010120
:1023F0005F0EEC6F0101020EA8DA01015E0EEC6FB8
:10240000F0DADADA0F0EA1DA0101610E99DA08C109
:10241000ECF10101010E99DA09C1ECF10101020EA2
:1024200094DA0AC1ECF1DDDA0BC1ECF10101040E22
:102430008CDA0CC1ECF10101050E87DA0DC1ECF16B
:102440000101060E82DA0401006B080E005D0AE24B
:102450000101EC69080E04010025010176DA04018E
:10246000002BF3D70101440E94DA0101440ED46F1E
:102470000101220E65DA70DA0D0EEB6FE9D9120058
:102480000101ED6BF0D9040B01E0000C010C01011E
:10249000010EEC6F010176DA120E52DAD7C1ECF1BF
:1024A0000101100EA5EF14F0010E0101DA150B6EFB
:1024B0000C6ADA510B240401D66F0101DB510C20A8
:1024C0000401D76F0101400E64DAD6C4ECF10101BA
:1024D0000A0E3BDAD7C4ECF101010B0E36DA01012A
:1024E000120EEC6F0101EB6BB3D90101DAC10BF0F5
:1024F000DBC10CF0DA07000EDB5B3FDA0DE2D8C17E
:10250000E9FFD9C1EAFFD82B000ED923EFCFECF1B8
:102510000101100EEB6FE8D7DA69DB6BDA51DB11E2
:1025200008E016DA400B05E10101DA07000EDB5B7B
:10253000F5D712000101010EEC6F010123DA0A0E3A
:10254000FFD90101100EE3EF14F0DEC137F4DFC153
:1025500038F40101400E1DDA37C4ECF101010A0E16
:10256000F4D938C4ECF101010B0EEFD901010A0EC8
:10257000E7D90101DEC10BF0DFC10CF0DE07000E70
:10258000DF5BFBD910E20101100E1DDAE66E0101DE
:10259000DCC1E9FFDDC1EAFFDC2B000EDD23E552E3
:1025A000E750EF6EE6D737C4F3FF38C4F4FF1200EC
:1025B0000101E051BBD9EE52EF6A12000101E15175
:1025C000B5D9EE52010EEF6EE1C1D6F11200010154
:1025D000D4050401376FE8500B6E0C6A0C50000AEA
:1025E000E8AE02D0D89004D0440E0B5C000E0C581C
:1025F00002E25E0E376FDCD937C4ECF1F1EF14F074
:10260000EBD90401006FD4D90101D5510401005D5B
:1026100007E25F0E0101D880D5550401002504D0E2
:102620000101D5510401005D016FE8500B6E0C6A89
:102630001B0ED8800B56000E0C560BC001F40BC0BD
:1026400003F4026B02C4F3FF0BC0F4FF120001019C
:10265000E00E76D90101030EB6D90401006FA8D9A6
:1026600004010051040B01E0000C010CE4C1E9FF7E
:10267000E5C1EAFFEF686CD9100B0FE00101210EF4
:102680005FD90101F0690DD967D97CD99FD990D95B
:102690009EDF92D90D0E59D9000C9ED90401126FFC
:1026A00087D90101D4510401125D58E0D4C114F45A
:1026B000136B13C4EEF1D4C1EFF1E1D8120E010196
:1026C000DE6FDF6B0101000EDC6F040EDD6F3DDF9E
:1026D00004010051010B3DE0400E025D000E035964
:1026E00038E3EE0ED8800255050E035532E310C4D0
:1026F000F3F011C4F4F015EC23F0F3CF10F4F4CFA1
:1027000011F4060EE66EE66A0A0EE66E040EE66E3A
:10271000E2C1E9FFE3C1EAFFE2C10BF0E3C10CF063
:10272000E2C1E6FFE3C1E6FF7AEC24F0F56E060EA7
:10273000E15EF550080E0401115D0BE1105103E05C
:10274000060E105D06E1E4C1E9FFE5C1EAFF10C431
:10275000EFFFD4C1D5F101C4D4F1010C000C01018B
:102760000A0E17D90101D651E1D8EFCFD4F40401F4
:10277000D36BD3C4EEF1D4C4EFF181D8060E0101BE
:10278000DA6FDB6BE6C1D8F1E7C1D9F18DDE08C1A4
:10279000D7F17DDE09C1D7F17ADE0AC1D7F177DE44
:1027A0000BC1D7F174DE0CC1D7F171DE0DC1D7F1C9
:1027B0006EDE0101E85103E10401D56B03D0040191
:1027C000060ED56F0101080ED76F61DED5C4D7F1B3
:1027D0005EDE0E0E0101E927000EEA233C0EE95DE4
:1027E000000EEA5903E2400EE96FEA6BE9C1D3F447
:1027F000EAC1D4F4E9C1ECF10101050EA6D8D4C4B4
:10280000ECF10101060EA5EF14F0C8D8240E98D8FB
:102810000401B16BB151AAD80AE2B15187D8EE5286
:10282000EF5003E0B1C4D6F11200B12BF3D7120080
:102830009568816AE00E936EF19E84828480848420
:10284000966A050EE66EBDEC26F0E5528494120001
:10285000EBC181FFE00E936EECC183FF956A849219
:102860008482956812009568EDC181FFE00E936E39
:10287000849083CFD8F484800401D8511200EEC133
:10288000D6F4EFC1D7F40101400E83D8D6C4ECF1E1
:102890000101080E5AD8D7C4ECF10101090EA5EFC9
:1028A00014F0F0C116F40401156B15C40BF016C436
:1028B0000CF01507000E165B60D8F7E31200D5C1C7
:1028C00014F40401120E136F0101F15104011327D6
:1028D0000101F2510401142313C4EEF114C4EFF109
:1028E0003FEF14F0F3C1D6F10101D6511FD8EFCF5D
:1028F000B2F404010E0EB16F0101F4510401B127CD
:102900000101F5510401B223B1C4EEF1B2C4EFF1FB
:102910003FEF14F00101090E56D80401016F0101C7
:10292000080E51D8F36E01C4F4FF1200E96EEA6A92
:10293000D890E936EA36D20EE926010EEA221200D4
:10294000EC6F0101EB6B28EF14F0EB6F28EF14F044
:102950000101070EE3EF14F00101EC6B010112001D
:102960000A0EE66E9FEC26F0E55212000B6E0C6A22
:10297000010E0B5C000E0C581200D8800B54000E98
:102980000C5412000A0EE1DFE7DF0B0EDEDF01015F
:102990001200EC6F0101070EA5EF14F00101D651F2
:1029A000C5DFEFCFECF10101040ECFDF0101120012
:1029B0000101200EA0EF14F00101EC690101070EE6
:1029C000C4DFACEF14F0ED6F33EF14F0020EEC6FD8
:1029D00001010D0EA5EF14F00101600EB1DFA8EFAB
:0A29E00014F00101030EA5EF14F03E
:0629EA00070E0201B05DC2
:1029F00001E11200FF0EB15D01E0B7DA0201B16939
:102A0000B06BB36B12000201B051060A01E1A6D00F
:102A1000030A67E0010A5AE0070A45E0010A32E0CA
:102A2000030A28E0010A01E01200040100690169BB
:102A30000269036904690569066907690869096922
:102A400002013A6B3B6B3C6B3D6B430E0101C36F64
:102A5000C46B0101000EC16F040EC26F440E010170
:102A6000BF6FC06BE0EC17F00201B16F5CDA0201DE
:102A7000010EB06F43DA140E64DA01E280D0020175
:102A8000020E3DD002013A513B113C113D1135E19E
:102A9000B1C2BEF140EC12F0000971E00201010E7A
:102AA00070DA030E2CD02ADAC80E4BDA03E30201E7
:102AB000020EB06FB1C2C7F1D1EC18F000095FE0AF
:102AC00064D802085CE10201040EB06FB1C2BEF12D
:102AD00040EC12F0000953E00201030E52DA050E39
:102AE0000ED0B1C2C7F1D1EC18F000092FE04DD8DB
:102AF00004010A6F060E0A5D04E10201040EB06FC4
:102B00001200050E0A5D29E130DA0201B1690BDA23
:102B10000201060EB06F3AC204F13BC205F13CC29D
:102B200006F13DC207F142C20EF143C20FF144C2A9
:102B300010F145C211F13EC212F13FC213F140C281
:102B400014F141C215F1B281B32B1200D7D9C80ECE
:102B5000F8D915E30201020EB06F1200CFD9640E4E
:102B6000F0D90DE33607000E375B385B395B365121
:102B700037113811391102E10201B06BD4D91200BA
:102B80000201080EB06FB5EF17F004010D6B0201E2
:102B90003C0E366F376B386B396BAAD9020E0401C5
:102BA0000B5D01E0E2D00C6B0F0E0C5D02E2F7D979
:102BB000FBD701013A0EC86F020EC0D93B0EC86F99
:102BC000020EBCD93C0EC86F020EB8D93D0EC86FBC
:102BD000020ED4D904010C6B080E0C5D02E2DFD9A1
:102BE000FBD70C6B060E0C5D0EE282D904010C5172
:102BF000EA6A080FE96E010EEA22EF500B5D01E070
:102C0000D6D00C2BEFD70C6B0C510B6E0C6A0C5002
:102C1000000AE8AE02D0D89004D0CE0E0B5C000EB5
:102C20000C5802E2BCD9F0D70E6B62D904010B51EB
:102C3000330A62E0CC0A5DE0C90A47E0350A23E0C6
:102C4000020A0DE0340A01E07DD052D904010B05DF
:102C500001E0ADD001010D0EC86F040E48D089D936
:102C600001E0A5D00101420EC86F020E67D9430EE4
:102C7000C86F020E63D9440EC86F020E5FD9450EAD
:102C8000C86F020E34D075D901E291D001013E0E19
:102C9000C86F020E53D93F0EC86F020E4FD9400EB7
:102CA000C86F020E4BD9410EC86F020E67D9040ED1
:102CB00004010B5F04010B510B07000952E00101F5
:102CC0000C0EC86F040E5AD9F5D753D970E1010123
:102CD000120EC86F040E32D9110EC86F040E2ED911
:102CE000100EC86F040E2AD90F0EC86F040E46D9F5
:102CF00038D0010E0E6F35D03CD959E10101390EA3
:102D0000C86F020E1BD9380EC86F020E17D9370EC6
:102D1000C86F020E13D9360EC86F020E2FD9080ED7
:102D2000D88002013655070E3755000E3855000E73
:102D3000395517E2080E365F070E375B000E385B19
:102D4000395B0FD001010B0EC86F040E17D90401B7
:102D50000B510B07000905E001010C0EC86F040EB2
:102D6000F5D704010E5101E160D7020E0D5D09E1B6
:102D70000FC432F210C433F211C434F212C435F26B
:102D800011D0320EE96E020EEA6EEE500F1908E114
:102D9000EE50101905E1EE50111902E1EE50121932
:102DA00001E00D6B02EC19F004010D51120002EC70
:102DB00019F0000C0101010EB1D8010EAFD8060EBA
:102DC000ADD8C7D8120EAAD8230EA8D8340EA6D8CC
:102DD000560EDCD8800EDAD8BCD8BBD8C66B32EC25
:102DE00018F004010B6B0C0E0B5D02E2B7D8FBD799
:102DF00008C1C6F132EC18F009C1C6F132EC18F086
:102E00000AC1C6F132EC18F00BC1C6F132EC18F071
:102E10000CC1C6F132EC18F00DC1C6F132EC18F05D
:102E200004010B6B0B510B6E0C6A0C50000AE8AEE0
:102E300002D0D89004D0CA0E0B5C000E0C5802E2EF
:102E40008DD8F0D70101630E69D8820E67D8530E72
:102E500065D8630E63D8350E61D8010EC66F32ECAB
:102E600018F04AC2C6F132EC18F002014A0518E027
:102E70003A513B113C113D1113E00101360E8AD845
:102E800035C2C6F132EC18F034C2C6F132EC18F09B
:102E900033C2C6F132EC18F032C2C6F132EC18F08F
:102EA0000101370E3BD8020E39D8010E37D8030E78
:102EB000C66F32EC18F0030E02014A5D13E1010106
:102EC000320E68D83AC2C6F132EC18F03BC2C6F1F5
:102ED00032EC18F03CC2C6F132EC18F03DC2C6F13B
:102EE00032EC18F00101C66932EC18F072EF18F0FC
:102EF00001010B0EC86F040EBEEF17F084EC26F034
:102F000002014651045C0B6E475105580C6E485146
:102F100006580D6E495107580E6E1200C66F32ECFE
:102F200018F00101120084EC26F004C046F205C03E
:102F300047F206C048F207C049F212001FD801014B
:102F400012000B5C000E0C58000E0D58000E0E58AF
:102F50001200C66B32EC18F0010112000101C66BC1
:102F600032EC18F004010B2B1200B1C2C5F12EEFA8
:102F700018F0BEDF040E04010B5D1200C96FDBEF19
:102F800018F04A6F17DFCFDF02011200C7DFE1DF61
:102F9000A9EF17F0C3DF040EC66F32EF18F0A8DFF9
:062FA00004010C2B1200DD
:0A2FA6000401006B020E005D07E25B
:102FB00000516FDA005165DAEF90002BF6D712005E
:102FC0000401920E0C6F010E0D6F0B6B020E0B5D68
:102FD00044E22ADA0C0E63DAEFCF0CF00D6A0E6AC7
:102FE0000B500C100D100E1032E11EDA0C0EBFC18A
:102FF000EBFF0D0EC0C1EBFF0101C151C21111E089
:103000000A0EE66EE66AC1C1E6FFC2C1E6FF0CDA4F
:103010000CC40BF00DC40CF00CC4E6FF0DC4E6FFAD
:1030200017DA02DA0A0EC3C1EBFF0B0EC4C1EBFFC5
:10303000FBD90E0EEB6A0F0EEB6AF6D9100EEB6A97
:10304000110EEB6A0BC4BEF104010B511200160EF7
:103050000C27000E0D230B2BB9D7FF0C0101C55116
:1030600049EF1AF00101BE51160DF3CFE9F4F4CF88
:10307000EAF4920E0401E927010EEA2306DAEE5083
:10308000ED100FE1C2D9120ED6C1EBFF1C0E0101EB
:10309000F46FF56BBAD9E3D9B8D9130EEB6A140EF5
:1030A000EB6AC6C1D7F147EC12F0AFD9130EF7D9CE
:1030B000EDCF0CF0EE2AEF22E8D9C4D90B5C0E500C
:1030C0000C5803E3E2D9EE2AEF22DFD9EECFEBF47E
:1030D000EDCFECF40401D60EEB5D030EEC5901E3E9
:1030E00001D8010C0101BE51160DF3CFE7F4F4CF66
:1030F000E8F4920E0401E727010EE8238BD90C0EA9
:1031000080D9B3D9F3CFDFF4F4CFE0F483D90A0E3A
:1031100078D9ABD9F3CFE1F4F4CFE2F47BD90E0E3A
:1031200070D9EECFE3F4EFCFE4F4080E0401E32707
:10313000000EE423E56BE66B140E0101F46FF56BF2
:1031400069D98DD9E3C49DF2E4C49EF20201110E47
:103150009C6F60D9E7C49AF2E8C49BF20AEC1BF0BA
:10316000E3C4F3F0E4C4F4F015EC23F0F3CFE3F49C
:10317000F4CFE4F4080E0101DA6FDB6B0101DF0E1E
:10318000D86F040ED96F54EC12F005EC14F042D94C
:10319000120E37D9EF683ED90E0EEB6A0F0EEB6AAE
:1031A0001200C7C1BEF167D9D880EE54000EED54AD
:1031B00001E3000C010C5FD9EE50ED1001E1000CB1
:1031C000BE515FD9EF50010B09E0BE515AD9EF90C3
:1031D0001C0E0101F16FF26B5FEC14F09AEC12F02F
:1031E000C8C1E9FFC9C1EAFFEF6E45D9EE06EF5A43
:1031F000BE51FDD8100E05D9EE50ED1002E1E7ECFE
:1032000012F0010C38D9EE50ED1002E0E7EC12F0AC
:1032100032D9EE6AED6A1200080E0101DE6FDF6B33
:103220000101000EDC6F040EDD6FA5EC12F000C48E
:10323000F3F001C4F4F015EC23F0F3CF00F4F4CF75
:1032400001F402C4F3F003C4F4F015EC23F0F3CF5F
:1032500002F4F4CF03F404C4F3F005C4F4F015EC65
:1032600023F0F3CF04F4F4CF05F40401080E045F57
:10327000000E055B06C4F3F007C4F4F015EC23F070
:10328000F3CF06F4F4CF07F4CAC1D0F1CBC1D1F12A
:103290000101000ECE6F040ECF6F14D80401086F29
:1032A000FF0E085D03E1E7EC12F0010C08519FD816
:1032B000100EA7D804C4EEFF05C4EDFF0851E1D8F5
:1032C000EF80010C04010A69920E0B6F010E0C6F66
:1032D000096B020E095D5BE2A2D80C0E92D8A9D848
:1032E000020E8FD8AFD80B184BE10E500C1848E1E6
:1032F00096D80A0E86D89DD8A5D80B183FE10E5057
:103300000C183CE18CD8100E7CD8EECF0FF0EFCF2C
:1033100010F0116A126A0F501010111012102EE1E5
:10332000D0C1E9FFD1C1EAFF060EB9D8EECF0CF04B
:10333000EECF0DF0EFCF0EF072D8060E62D8EE5041
:1033400000010B1908E1EE500C1905E1EE500D19C2
:1033500002E1EE500E190FE062D8060E52D8E8686E
:10336000EE180CE1E868EE1809E1E868EE1806E1ED
:10337000E868EE1803E104010951120009C40AF4D7
:103380000401160E0B27000E0C23092BA2D7FF0EEB
:103390000A5D2AE00A51160DF3CF0BF4F4CF0CF4BA
:1033A000920E0B27010E0C230A0EE66EE66AD0C1C0
:1033B000E6FFD1C1E6FF33D80BC40BF00CC40CF010
:1033C0000BC4E6FF0CC4E6FF43D8CEC1E9FFCFC172
:1033D000EAFFEECF0BF0EFCF0CF021D80A0E0BC0B6
:1033E000EBFF0B0E0CC0EBFF04010A511200160D8F
:1033F000F3CFE9FFF4CFEAFF920EE926010EEA22AD
:103400001200E926000EEA221200E9C4E9FFEAC42C
:10341000EAFF1200E7C4E9FFE8C4EAFF12000BC4A8
:10342000E9FF0CC4EAFF12000CC4E9FF0DC4EAFF77
:103430001200EECF0BF0EFCF0CF0CEC1E9FFCFC101
:10344000EAFF1200EECF0DF0EFCF0EF00D5012009C
:103450007AEC24F0F56E060EE15EF5501200120EC5
:10346000EB500101F36F72EF14F0EECFF3F0EDCFFC
:10347000F4F015EF23F00101BE51B9DF100E01EF9A
:103480001AF0B5DF150E01EF1AF0BFDF0E0E01EFD7
:103490001AF0ADDF0C0EB5DFEE6AED6A1200B1DF97
:0634A000EECF0BF012005C
:0A34A600140E0101DE6FDF6B01015F
:1034B000080EDC6F040EDD6FA5EC12F0F00E0401B7
:1034C0000815400801E0A3D00F0E0815040DF350B5
:1034D0000B6E0C6A140E0B5E000E0C5A0BC01CF423
:1034E0000B50140801E293D01C5100080BE21C5150
:1034F0000101DE6FDF6B01011D0EDC6F040EDD6F5D
:10350000A5EC12F012C400F413C401F40401126B10
:10351000136B140E17D9080EF96F040EFA6F4EECE8
:1035200023F0F3CF04F4F4CF05F40401041F051FC6
:103530001C51000810E21C5105D91D0EF96F040E34
:10354000FA6F4EEC23F0F3CF06F4F4CF07F4040146
:10355000061F071F02D0066B076B040EF3D8040E7C
:10356000F96F040EFA6F4EEC23F0F3CF02F4F4CFB0
:1035700003F40201080E9F6F040EA06FBCD8040173
:103580000251001944E10351011941E1F00E0815FF
:1035900040083DE10201925193110CE092C2E9FF13
:1035A00093C2EAFF18C4EEFF19C4EEFF1AC4EEFF7F
:1035B0001BC4EEFF94C2E9FF95C2EAFF060EE9269E
:1035C000000EEA2214C4EEFF15C4EEFF16C4EEFF8F
:1035D00017C4EEFF96C2E9FF97C2EAFF11C4EFFFDE
:1035E00004011C510D6E0E6A0D500A5D0B6E0E50DB
:1035F0000B590C6E140E0B5E000E0C5A98C2E9FFAC
:1036000099C2EAFF0BC0EEFF0CC0EDFF010CE7EC26
:1036100012F0000C0401450EB16FB26B140E0201E2
:103620009D250401B36F000E02019E210401B46FB9
:103630000001FD2B000EFE23FDC0B5F4FEC0B6F464
:103640000401B76BB86B640EB96F9CC2BAF4BB6B64
:10365000BC6B04C1BDF405C1BEF406C1BFF407C113
:10366000C0F49AC2E9FF9BC2EAFF060EE926000EEB
:10367000EA22EECFC1F4EECFC2F4EECFC3F4EFCF27
:10368000C4F40201B10E9F6F040EA06F34D8140E63
:1036900059D8B10EF96F040EFA6F4EEC23F0F3CF48
:1036A000BBF4F4CFBCF4140E02019D250101E96FB7
:1036B000000E02019E210101EA6F0101E86B9AC22E
:1036C000E9FF9BC2EAFF9AC2E6F19BC2E7F1AFECC9
:1036D00013F0140E0101DA6FDB6B0101B10ED86F2C
:1036E000040ED96F54EC12F00B6A0C6A0BC0F3FF96
:1036F0000CC0F4FF12002FD8020E15D8020EF3CF23
:10370000EBFF030E24D8040E0ED8040EF3CFEBFF0C
:10371000050E1DD80A0E07D80A0EF3CFEBFF0B0ECD
:103720000CC0EBFF1200E926000EEA22EECFF3F008
:10373000EDCFF4F015EC23F0F3CF0BF0F4CF0CF059
:10374000ABEF1BF00001FB6FFC6B000112000CC023
:10375000EBFFABEF1BF09FC2E9FFA0C2EAFF120034
:103760001C0E0101DE6FDF6B0101000EDC6F040E29
:10377000DD6FA5EC12F0E7EC12F00201000EA86F6D
:10378000040EA96FF5D80401010E001912E10151D0
:1037900010E104510B6E0C6A060E0B180AE10C5076
:1037A00008E105510D6E0E6A040E0D1801E10E5070
:1037B00001E0000C020E061905E1075103E106D9EC
:1037C000EF6A0DD0010E061906E1075104E1010E62
:1037D000FDD8EF6E04D0020EF9D8EF6E000C010197
:1037E00004510401185D2EE1010105510401195D28
:1037F00029E10101065104011A5D24E1010107518B
:1038000004011B5D1FE1A1C2E9FFA2C2EAFF08C4D7
:10381000EEFF09C4EEFF0AC4EEFF0BC4EEFF0CC4BA
:10382000EEFF0DC4EEFFA1C2E9FFA2C2EAFF060E41
:10383000D7D80EC4EEFF0FC4EEFF10C4EEFF11C4C4
:10384000EEFF010C000C010E0401006F016B026B16
:10385000080E036F060E046F040E056F0201A70524
:103860000BE1010E0401066F076B126913691469FD
:1038700015691669176914D0020E0401066F076BEB
:10388000A5C2E9FFA6C2EAFFEECF12F4EECF13F411
:10389000EECF14F4EECF15F4EECF16F4EFCF17F40D
:1038A00008C108F409C109F40AC10AF40BC10BF4F8
:1038B0000CC10CF40DC10DF404C10EF405C10FF4DC
:1038C00006C110F407C111F47AD8EF500E190101A6
:1038D0000E151BE174D8010E83D8EF5004010F19A7
:1038E00001010F1512E16BD8020E7AD8EF500401D6
:1038F00010190101101509E162D8030E71D8EF50BB
:10390000040111190101111509E012C118F413C1C4
:1039100019F414C11AF415C11BF409D050D8EECF14
:1039200018F4EECF19F4EECF1AF4EFCF1BF4020126
:10393000000EA86F040EA96F1BD81C0E0101E96FC1
:10394000EA6B0101060EE86F0101120EE66F040E2C
:10395000E76FAFEC13F01C0E0101DA6FDB6B0101B6
:10396000000ED86F040ED96F54EC12F005EF14F06E
:1039700032D819D8F3CFEEFF0CC0EDFF2CD8020ED1
:103980002FD811D8020EF3CFEBFF030E0CC0EBFFC4
:1039900022D8060E25D807D8060EF3CFEBFF070E68
:1039A0000CC0EBFF1200EECFF3F0EDCFF4F015EC0E
:1039B00023F0F3CF0BF0F4CF0CF0EBEF1CF0A5C22B
:1039C000E9FFA6C2EAFF060EF0EF1CF0A3C2E9FF72
:1039D000A4C2EAFF1200A8C2E9FFA9C2EAFF1200CE
:0839E000E926000EEA221200A4
:0839E8000201836B826B0201F6
:1039F0000B0E726F17EC1FF0010C020182A103D0B5
:103A00000B6A0C6A63D0200E04014C6F4D6B89C2A7
:103A1000E9FF8AC2EAFFEF5057E0F5D8FFEC24F047
:103A2000E552E552F3CF89F2F4CF8AF202010F0E8C
:103A30007F6F02013D0E7D6F040E7E6F4CC47BF2E2
:103A40004DC47CF20201A00E7A6FB7EC1FF00401A6
:103A50003D512EE1D8D8C6EC24F0E552E552F3CF23
:103A60004EF40401F3500C0802E20C0E4E6F4E515E
:103A7000E66EE66A400EE66E040EE66EC4D8D4EC3E
:103A800024F0F56E060EE15EF55000090BE13EC430
:103A900086F23FC487F20201832B3EC4F3FF3FC48A
:103AA000F4FF12000F0E04014C27000E4D23BED769
:103AB000040E3D5D09E13E1D01E13F1D05E03EC4F0
:103AC0004CF43FC44DF4B2D70B680C680BC0F3FF45
:103AD0000CC0F4FF12000201886B8291835101E057
:103AE000830712008BC284F28CC285F28BC277F2FC
:103AF0008CC278F20201A00E766F58EC1FF000091C
:103B000001E0000C010C71D8030E0401D35D02E149
:103B10006CD806D0040ED35D03E102018469856987
:103B20000401D3511200ACEC1FF068D00201828175
:103B3000200E0C6AF36E0CC0F4FF12008DC284F2EA
:103B40008EC285F28DC288F23F0E020188178DC2A7
:103B500074F28EC275F20201A00E736F22EC1FF098
:103B6000000901E0000C010C8FC279F285EC1FF016
:103B7000000901E0000C0201882B842B000E852334
:103B8000400E885D0AE30AD884C274F285C275F2D9
:103B90000201A00E736F22EC1FF0010C0201886B72
:103BA00099EC1FF00201A00E806FE6EC1FF00009F7
:103BB000F9E124D086C28BF287C28CF293DF040134
:103BC000C96BCA6B0401C9C40BF0CAC40CF0C92B81
:103BD000000ECA23020190510B1802E191510C18FA
:103BE00002E091DFEFD79FDF09D0A3EC1FF00401C3
:103BF000D36F0201842B000E8523120084C2F3FFD1
:103C000085C2F4FF120089C2E6FF8AC2E6FF1200F5
:103C1000FF0EE3CFEAFFE552FF0EE3CFE9FFE552E7
:103C2000E66AE66AD9CFE6FFDACFE6FFFC0EE124CA
:103C3000D96EFF0EE220DA6EE66AE66AE66A200EC8
:103C4000EF5C06E0090EEF5C03E0EF6603D03FD0C7
:103C5000EE50F5D72D0EEF5C03E1FF0EE32A03D003
:103C60002B0EEF5C01E1EE502F0EEF6424D03A0EE4
:103C7000EF6021D0D890F90EE336FA0EE336FD0E50
:103C8000DECFE3FFFE0EDDCFE3FFD890F90EE33683
:103C9000FA0EE336D890F90EE336FA0EE336FD0E4F
:103CA000E350DE26FE0EE350DD22300EEE5CDE2613
:103CB000000EDD22D9D7FF0EE3CFE8FFE85207E080
:103CC000F90EE31EE32AFA0ED8B4E306E31EE5522A
:103CD000E552E552FF0EE3CFDAFFE552FF0EE3CFE8
:103CE000D9FFE552E1CFE9FFE2CFEAFFED52ED5215
:103CF000EECFF3FFEFCFF4FF1200D9CFE6FFDACF1C
:103D0000E6FFFA0EE3CFD9FFFB0EE3CFDAFFFD0E9D
:103D1000E35209E72D0EDE6EFC0EE31EE32AFD0ED4
:103D2000D8B4E306E31EE652E652E652FD0EE12465
:103D3000E76EFF0EE220E46EE652F70EE3CFE6FFF9
:103D4000F70EE3CFE6FFEDEC1EF0F90EE124E96E8D
:103D5000FF0EE220EA6EDDEC1EF00AE1DAEC1EF066
:103D600009E1DDEC1EF008E1DAEC1EF007E108D015
:103D7000E8EC1EF0E3EC1EF0E8EC1EF0E3EC1EF0C5
:103D8000E8EC1EF0DE6AF90EE126FF0EE222FF0EDD
:103D9000E3CFDAFFE552FF0EE3CFD9FFE552FC0E89
:103DA000E124E96EFF0EE220EA6EEECFF3FFEFCFE3
:103DB000F4FF1200EF380F0B1200EF500F0B02E16F
:103DC000EE52D8841200EF380F0B300FDE6E120067
:103DD000EE500F0B300FDE6E1200FC0EE3CFE9FF4A
:103DE000FD0EE3CFEAFF100EE66EEE6AEE6AEF6AB2
:103DF000D890FD0EE336FE0EE336ED36ED36EF36A7
:103E0000FF0EE30609E00EEC1FF0EE520EEC1FF081
:103E1000EE520EEC1FF0EDD7E56E1200030EEF240C
:0E3E2000E8B6EF6E300EEF24E8BEEF6E000C39
:023E2E003F0E45
:103E3000C716C66AC56AC68694869488C68A72C240
:103E4000C8FF120074C2D3F475C2D4F4C750040B77
:103E500001E0010EEFD8FAE1C580C5B0FED7A1B6EA
:103E6000010C73C281F2EBD801E0010CC750040BC6
:103E700001E0010EDFD8FAE1C5BC19D0D4C481F24B
:103E8000DED801E0010CC750040B01E0010ED2D8CE
:103E9000FAE1D3C481F2D3D801E0010CC750040B7E
:103EA00001E0010EC7D8FAE1C5AC000C020C020C0F
:103EB00077C274F278C275F276C273F2C3DF04017E
:103EC000D56FE85005E176D80401D56FE85002E0DF
:103ED000D5511200C750040B01E0010EABD8FAE136
:103EE000C580C5B0FED7A1B6010C0201762902013A
:103EF000816FA5D801E0010CC750040B01E0010E51
:103F000099D8FAE1C5AC000C020CC750040B01E0D3
:103F1000010E90D8FAE179C281F291D801E0010C4A
:103F2000C750040B01E0010E85D8FAE1C5AC000CC6
:103F3000020CC750040B01E0010E7CD8FAE1C584E5
:103F4000C5B4FED7000C71D8C5B6FED7C59AC588D2
:103F5000C5B8FED7C950120068D8C5B6FED7C58A05
:103F6000C588C5B8FED7C584C5B4FED7000C7BC2D2
:103F700077F27CC278F27AC276F29ADF0401576F48
:103F8000E85016E102017F517F0700090EE0DBDFF8
:103F9000E66E02017DC2E9FF7EC2EAFF7D2B000EC4
:103FA0007E23E552E750EF6EEDD7D6DF0401576F61
:103FB00057511200C750040B01E0010E3BD8FAE143
:103FC000C584C5B4FED7A1B6010C000CC750040BC4
:103FD00001E0010E2FD8FAE1C580C5B0FED7A1B629
:103FE000010C80C281F22BD801E0010CC750040BF8
:103FF00001E0010E1FD8FAE1A1B6010CC5BC03D047
:104000000401A96B03D00401040EA96FC584C5B4D3
:10401000FED7A1B6010C0401A951120081C2C9FF4B
:10402000C6BEFF0CC7B0FED7000CC586C7A0FED722
:10403000C95012000B6E1F0EC5140B101200EEDFDC
:044040000009120061
:0C404400080E0101DE6FDF6B0101000EB1
:10405000DC6F040EDD6FA5EC12F002C42EF403C475
:104060002FF40401026B036B080E0001FB6FFC6B65
:104070000001000EF96F040EFA6F4EEC23F0F3CF3F
:1040800028F4F4CF29F40401281F291F080E0B6E11
:10409000D9D8E850EF5ED6D8EF500101DE6FDF6B64
:1040A0004DC2DCF14EC2DDF1A5EC12F0CBD8EF50E1
:1040B0000001FB6FFC6B4DC2F9F04EC2FAF04EEC02
:1040C00023F0F3CF2AF4F4CF2BF404012A1F2B1F83
:1040D000040E0001FB6FFC6B0001280EF96F040E4B
:1040E000FA6F4EEC23F0F3CF2CF4F4CF2DF4020151
:1040F000000E5F6F040E606F7AD84BC2E9FF4CC2AE
:10410000EAFF00C4EFFF51C2E9FF52C2EAFF04C454
:10411000EEFF05C4EDFF53C2E9FF54C2EAFF06C437
:10412000EEFF07C4EDFF04012E512C1902E12F51BF
:104130002D1901E0000C010C0401016B57C200F4C1
:10414000026B036B5BC204F45CC205F45DC206F44F
:104150005EC207F402015A51E66EE66A58C2E6FFF3
:1041600059C2E6FF080EE66E040EE66E7AEC24F005
:10417000F56E060EE15EF5500201000E5F6F040E53
:10418000606F35D8080E02015A250001FB6FFC6BE9
:10419000000EFC230001000EF96F040EFA6F4EECC6
:1041A00023F0F3CF02F4F4CF03F4080E02015A25F2
:1041B00002019D6F9E6B000E9E230201010E9C6FFB
:1041C00055C29AF256C29BF20AEC1BF0080E02018D
:1041D0005A250101DA6FDB6B000EDB230101000EB3
:1041E000D86F040ED96F54EC12F005EF14F02FD8ED
:1041F000040E15D8040EF3CFEBFF050E1FD8060EE4
:104200000ED8060EF3CFEBFF070E18D8020E07D814
:10421000020EF3CFEBFF030E0CC0EBFF1200E926FA
:10422000000EEA22EECFF3F0EDCFF4F015EC23F020
:10423000F3CF0BF0F4CF0CF027EF21F00CC0EBFF25
:1042400027EF21F04FC2E9FF50C2EAFF12005FC220
:08425000E9FF60C2EAFF120061
:0842580044656D6F534E4D509B
:1042600020312E3000444843502F476C65616E6901
:104270006E672E2E2E00426F617264205365747536
:10428000702E2E2E002020202020202020202020D4
:104290002020202020000D0A0D0A0D4D43485053C8
:1042A0007461636B20534E4D50204167656E7420DE
:1042B00044656D6F204170706C69636174696F6EE5
:1042C00020312E3020284D6963726F636869702039
:1042D0005443502F495020537461636B20322E3267
:1042E000302B205365702032342032303033290D8A
:1042F0000A0D0A09313A204368616E676520426FF2
:104300006172642073657269616C206E756D62659F
:10431000722E0D0A09323A204368616E6765206487
:10432000656661756C7420495020616464726573C0
:10433000732E0D0A09333A204368616E6765206465
:10434000656661756C742067617465776179206159
:104350006464726573732E0D0A09343A20436861F0
:104360006E67652064656661756C74207375626E36
:104370006574206D61736B2E0D0A09353A20456E08
:1043800061626C65204448435020262049502047F4
:104390006C65616E696E672E0D0A09363A204469B4
:1043A0007361626C652044484350202620495020A8
:1043B000476C65616E696E672E0D0A09373A2044B5
:1043C0006F776E6C6F6164204D50465320696D614C
:1043D00067652E0D0A09383A20536176652026203C
:1043E000517569742E0D0A0D0A456E74657220614F
:1043F000206D656E752063686F6963652028312DB7
:1044000038293A20000D0A496E76616C696420698A
:104410006E707574207265636569766564202D2001
:10442000496E7075742069676E6F7265642E0D0A2F
:10443000507265737320616E79206B657920746F9B
:0F44400020636F6E74696E75652E2E2E0D0A0047
:104450000201006B0181B4EC11F014EC25F0D3EFF4
:1044600017F00401010E366F0401365101E1D5D079
:10447000366B02010051040A01E1AFD0070A01E1E5
:1044800079D0040A65E0050A38E0070A2FE0050A3A
:1044900002E0010AE9E10101350EE46F040EE56F67
:1044A0000101020EE26F020EE36F36EC13F0000919
:1044B0000EE127EC13F00009D7E10101046B056B55
:1044C000066B076B02010181F5EC14F0CDD70401F6
:1044D000010E366F355103E10201020E33D0060E94
:1044E000355D01E077D00201050E2CD00401366B5A
:1044F00021EC25F00009B8E08DD002010C0E986F78
:10450000020E996F0201350E966F040E976F02012D
:10451000020E946F020E956F0201310E926F040E1F
:10452000936F53EC1AF0000910E00401010E366F8E
:10453000350503E10201030E05D0110E355D04E1DE
:104540000201070E006F90D7366BE7EC12F062D0D5
:104550000CC2CCF10DC2CDF10101020ECA6F020EE8
:10456000CB6F0CEC19F0000902E00201006B0401B2
:10457000366B7AD7006B290ED8800C55000E0D557E
:1045800029E30201300E536F020E546F02012E0E0A
:10459000516F020E526F02010C0E4F6F020E506FE0
:1045A00002010E0E4D6F020E4E6F0201350E4B6F63
:1045B000040E4C6F22EC20F000090AE0080E040102
:1045C000355D06E1010E366F0201040E006F02D068
:1045D0000201006BE7EC12F047D740EC12F0000943
:1045E00001E142D730C25DF231C25EF22EC25BF20F
:1045F0002FC25CF20CC25AF202010E0E586F020E6C
:10460000596F0201576B0201020E556F020E566F71
:104610009CEC20F00201006B27D703EC15F002019F
:0A462000B2A102D0020101911200C4
:06462A00F4C0F3FFF3C031
:10463000F4FF1200D9CFE6FFF5C001F4F6C002F492
:10464000F7C003F4F8C004F40401010E056F040E72
:10465000066F05C4E9FFEA6E030EA5D8EF50E66EBB
:10466000030E9BD800C4EFFF8FD8020E9CD8010E1A
:1046700090D8EF50E66E88D8020E8FD8010E89D8F8
:1046800000C4EFFF01C404F002C405F003C406F047
:1046900004C407F0E552E7CFD9FF12000401DB6B39
:1046A000DC6BDD6BDE6BFBC0D3F4FCC0D4F4D890C4
:1046B000D433D333F9C0D5F4FAC0D6F4D3C40BF055
:1046C000D4C40CF0D307000ED45B0B500C1018E0D0
:1046D000D5C4E9FFD6C4EAFF020ED527000ED623C3
:1046E000EECF0BF0EFCF0CF000010B510401DB27F4
:1046F00000010C510401DC23000EDD23DE23DED794
:104700000001FB51010B0EE0D5C4E9FFD6C4EAFF5E
:10471000EFCF0BF000010B510401DB27000EDC236F
:10472000DD23DE23DDC4D9F4DEC4DAF4DDC4D3F442
:10473000DEC4D4F40401D951DA111BE0DD6BDE6B69
:10474000DBC40BF0DCC40CF00D6A0E6AD3C40FF0AE
:10475000D4C410F0116A126A0B500F24DB6F0C5096
:104760001020DC6F0D501120DD6F0E501220DE6F17
:10477000D9D7DBC40BF0DCC40CF00B1E0C1E0BC035
:10478000F3FF0CC0F4FF120005C4E9FF06C4EAFF02
:104790001200E926000EEA221200FBDFE552E75084
:1047A000EF6EC4EF23F0F5DFEFCF00F4C4EF23F09A
:1047B000F00E83160F0E9512959A9598929A839AF9
:1047C0008398809ABFEC10F0F00E951687D8C5EC50
:1047D00010F0F00E83D8CBEC10F0F00E7FD80F0E57
:1047E00095120201280E76D8280E74D8080E72D8B9
:1047F0000C0E70D8010E6ED8130E6CD8800EAA6FF6
:1048000002EF24F014D80009FDE1959A9598F00E76
:10481000951683160201AA390F0B8312839A839887
:1048200052D8F00E83160F0E0201AA155ED0838AAD
:104830008398959A9598CBEC10F0808ACBEC10F089
:1048400083A604D0809A3FD8839A010C809A3BD8E3
:10485000839A000CABC2E9FFACC2EAFFEFCF0CF4C5
:10486000EF5008E00CC4AFF218D80201AB2B000ED9
:10487000AC23F0D71200ADC2F6FFAEC2F7FF0800BE
:10488000F5CF0CF4F55008E00CC4AFF206D80201E5
:10489000AD2B000EAE23EFD71200C9DF0009FDE1FA
:1048A000959A9598F00E951683160201AF390F0B65
:1048B0000F0B83128388839A06D8F00E83160F0E8F
:1048C0000201AF1512D0CBEC10F0808ACBEC10F0C7
:1048D000809A1200AA6F96DF02011200831683826B
:1048E000808ACBEC10F0809A12008312ECDF0F0E5E
:0448F000951212000B
:0C48F400D9CFE6FFDACFE6FFFA0EE3CFE3
:10490000D9FFFB0EE3CFDAFFFC0EE3CFE9FFFD0E8C
:10491000E3CFEAFFE9CFF3FFEACFF4FFF80EE3506D
:1049200003E1F90EE35008E0F80EE30602E2F90EA7
:10493000E306DECFEEFFF2D7FF0EE3CFDAFFE5525C
:10494000FF0EE3CFD9FFE5521200D9CFE6FFDACF51
:10495000E6FFFA0EE3CFD9FFFB0EE3CFDAFFFC0E42
:10496000E3CFE9FFFD0EE3CFEAFFE9CFF3FFEACFA4
:10497000F4FFDECFEFFFEE66FCD7FF0EE3CFDAFFEA
:10498000E552FF0EE3CFD9FFE5521200FE0EE3CF52
:10499000E9FFFF0EE3CFEAFFF36AF46AEE5203E0A9
:1049A000F34AF42AFBD71200D9CFE6FFDACFE6FFAD
:1049B000FA0EE3CFD9FFFB0EE3CFDAFFFC0EE3CF15
:1049C000E9FFFD0EE3CFEAFFF80EE35003E1F90E35
:1049D000E3500AE0F80EE30602E2F90EE306DE50C9
:1049E000EF5C02E1EE66F0D7F36EFF0EE3CFDAFF85
:1049F000E552FF0EE3CFD9FFE552F3501200FE0E51
:104A0000E3CFE9FFFF0EE3CFEAFFE9CFF3FFEACF01
:104A1000F4FF610EEF5C05E67B0EEF5C02E7DF0E54
:084A2000EF16EE52F6E1120060
:084A28000201616B6269636920
:104A30006469656966696769686B696B6A6B6B6BEA
:104A400012000201615129E10201260EA36F040E3A
:104A5000A46F02011C0EA16F040EA26FB0EC1BF03C
:104A600000092CE00401265115E11CC462F21DC4AA
:104A700063F21EC464F21FC465F220C466F221C44E
:104A800067F222C468F223C469F224C46AF225C41E
:104A90006BF2010C0201010E616F40EC12F0000993
:104AA0000CE00201A76B02011C0EA56F040EA66F9D
:104AB00023EC1CF00201616B010C000C010C6CC2B8
:104AC000E9FF6DC2EAFFEECF22F4EECF23F4EECF82
:104AD00024F4EFCF25F40201010EA76F02011C0E92
:104AE000A56F040EA66F23EF1CF06EC2E9FF6FC224
:104AF000EAFF02016851EE1808E16951EE1805E17C
:104B00006A51EE1802E16B51EE1814E001011251E6
:104B10000201685D20E1010113510201695D1BE1A1
:104B20000101145102016A5D16E1010115510201F2
:104B30006B5D11E170C2E9FF71C2EAFF62C2EEFF74
:104B400063C2EEFF64C2EEFF65C2EEFF66C2EEFF17
:084B500067C2EEFF010C000C2E
:084B58000D0A4E6F7720727503
:104B60006E6E696E67206170706C69636174696FE5
:104B70006E2E2E2E000D0A526561647920746F200E
:104B8000646F776E6C6F6164204D50465320696D81
:104B9000616765202D2055736520586D6F64656DC4
:104BA0002070726F746F636F6C2E0D0A000D0A44D3
:104BB000484350202620495020476C65616E696E3D
:104BC000672064697361626C65642E0D0A000D0ACA
:104BD00044484350202620495020476C65616E6947
:104BE0006E6720656E61626C65642E0D0A000D0AA9
:104BF00044656661756C74205375626E6574204DF2
:104C000061736B2028000D0A44656661756C742021
:104C100047617465776179204164647265737320BC
:104C200028000D0A44656661756C74204950204166
:104C30006464726573732028000D0A53657269619C
:104C40006C204E756D62657220280044656D6F534F
:084C50004E4D5020312E3000C2
:084C58002A0EF66E000EF76E45
:104C6000000EF86E01010900F550FB6F0900F550C8
:104C7000FC6F03E1FB6701D03DD00900F550F66FF2
:104C80000900F550F76F0900F550F86F09000900A9
:104C9000F550E96E0900F550EA6E090009000900B7
:104CA000F550F96F0900F550FA6F09000900F6CFC9
:104CB000FDF1F7CFFEF1F8CFFFF1F6C1F6FFF7C136
:104CC000F7FFF8C1F8FF0101F95302E1FA5307E0D9
:104CD0000900F550EE6EF907F8E2FA07F9D7FDC1C1
:104CE000F6FFFEC1F7FFFFC1F8FF0101FB07000E51
:064CF000FC5BBFD71200BF
:0A4CF6003C0ED66ED768070ED56E8F
:104D0000D58EF284F28A1200D9CFE6FFB4C204F045
:104D1000B5C205F0B6C206F0B7C207F0E552E7CF5C
:104D2000D9FF1200F2A40AD0D7683C0ED66E020159
:0E4D3000B42B000EB523B623B723F294120065
:024D3E00FF0E66
:104D4000E350136E480E01D04C0EE76EE72EFED7EF
:0E4D5000E76AE72EFED7132EF7D700001200F9
:024D5E0015EE50
:104D600000F025EE00F0F86A0A9CA68EA69C2CECBA
:0A4D700026F0C6EC0BF0FDD7120090
:064D7A00FF0EE350E84EBD
:104D80001200000000D000D000D0E82EFAD71200A8
:104D900002010202020404FF04FF40044104430430
:044DA000420406FFC4
:024DA40000000D
:044DA60000FF00000A
:044DAA000000000005
:024DAE0044655A
:104DB0006D6F534E4D5020312E30000000000C021C
:104DC00000000000000000000000000000000000E3
:104DD00000000000000000000000000000000000D3
:104DE00000000000394C224C064CEE4BCE4BAD4B34
:044DF000754B584B5C
:020000040030CA
:08000000FFFAFFFEFFFEFBFF0B
:00000001FF
